:040000008031A02883
:100008007E14803120007F08F0000C1621001B08A8
:10001800A0001C08A1009D14A11F1428A001A10183
:10002800A2012008A6072108A73D0030A83D260800
:10003800A9072708AA3D2808AB3D2908AC072A08C4
:10004800AD3D2B08AE3D2C08AF072D08B03D2E085E
:10005800B13DDC0A5C0882070000882863289428E0
:10006800DC0135082F02B8003608303BB9003708E4
:10007800313BBA0050083802BB005108393BBC007C
:1000880052083A3BBD0053083B02BE0054083C3BB3
:10009800BF0055083D3BC00057083F02A300580861
:1000A800403BA4003208B5003308B6003408B70056
:1000B8002F08B2003008B3003108B400992844086A
:1000C800D0004508D1004608D2003808C4003908D5
:1000D800C5003A08C6004708D3004808D4004908B4
:1000E800D5003B08C7003C08C8003D08C9004A08BD
:1000F800D6004B08D7004C08D8003E08CA003F0875
:10010800CB004008CC009928FF30A3027F30A43BE5
:100118005D18DD14DD1C9928230823009A0099280E
:10012800DD1C9928240823009A0020000C12911045
:100138007008FF007E1009008031A2289F308400DB
:10014800213085005130FE000030FF008731F22752
:100158008031FC0120308400003085003030FE0002
:100168000030FF008731F2277E1020008031BC2844
:10017800033023008C008D01463022009D002600AC
:100188008C018D018E01033021008C0020008C0130
:10019800813021008D0020008D0121008E014F301B
:1001A80020008E0030009101B1019201B20193014B
:1001B800B3019401B4019601B6019701B701980102
:1001C800B8019901B90101309A000130BA00013033
:1001D8009B000130BB0001309C000130BC00FF30A7
:1001E800A600FF30A5002300910192013F302000B6
:1001F800DB005B0823009505151413083000C500C3
:10020800003023009200013091003F302000DB00D5
:100218005B0823009505151413083000C6007F30CD
:10022800A400FF30A30046082000DC003000450889
:100238002000DB00DC36DB0C5B083000C30020004C
:100248005C083000C400A201C201A101C1019D01E6
:10025800BD019E01BE019F01BF01A901C901AA01FB
:10026800CA01AD01003023009200023091003F30F6
:100278002000DB005B0823009505151413082000F7
:10028800DB005B08E00060080F393000CD00AB01EF
:10029800CB01AC01CC010130AE000130CE00AF0182
:1002A800CF01A001C001013095000130B500C03078
:1002B8009100C030B100CC302000DB005B08210089
:1002C800940520000C16000020000C1296019701DE
:1002D800210091131110013020009800990122008B
:1002E8001D17210011110530250093002000111160
:1002F8008F31922780318F31732780318F31B0272A
:1003080080312000921F8A29921301008F31B02773
:100318008031E030F2008630F3008F31C027803121
:1003280020000C16000020000C123C30DB005B089B
:10033800F100A0308F31832780312100DC01FC01DE
:100348002000BE01BF018F31EA278031083020002C
:10035800DB005B08CA00FF30C4007F30C500CC0159
:100368002100DD01DD0AC73020009B0004309C001D
:10037800210091140B178B178F31A1278031200092
:10038800DB005B08E00060080319322A600884314A
:100398001A2480312000DB005B08E0006130600631
:1003A8000319D8292100DD0121005D08031D1D2A3C
:1003B8002030F2008730F3008F31C02780312000D1
:1003C80060088F316C2780313D308F316C27803148
:1003D80020006008DB00DC015B08FA005C08FB0019
:1003E80086313D2680318F317B2780311D2A2000C0
:1003F800CC0121005D14322A20006008042A7030E4
:10040800DB005B08CC00322A8F31EA278031322AA0
:100418008F31EA27803101302000B10080301B2A5B
:100428008F31EA278031FF302000B1007F30B200E1
:10043800322A20006008613A0319FB290C3A031993
:10044800142A033A0319002A1E3A0319032A023A06
:100458000319082A083A03190C2A322A2000111D08
:100468005F2B111185315C258031562B7C0A0319CD
:10047800532A2430F2008730F3008F31C0278031AF
:100488007C082000DB00DC015B08FA005C08FB004C
:1004980086313D26803120308F316C2780311C30E9
:1004A800F2008730F3008F31C027803120003F08E9
:1004B800FB003E08FA0086313D2680310830F20004
:1004C8008730F3008F31C027803120004F08FB00B0
:1004D8004E08FA0086313D2680310D30F200873013
:1004E800F3008F31C027803120002A08DB002B0859
:1004F800DC002C08DD002D08DE000430DF00DE37CC
:10050800DD0CDC0CDB0CDF0B832A5C08FB005B08D2
:10051800FA0086313D268031F630F2008630F3004D
:100528008F31C027803120004108FB004008FA00C5
:1005380086313D2680310230F2008730F3008F315A
:10054800C027803120003208FB003108FA008631CC
:100558003D268031FC30F2008630F3008F31C02711
:10056800803130002308013EFA008030243DFB0032
:1005780086313D2680311230F2008730F3008F310A
:10058800C027803121002108FB002008FA008631AD
:100598003D2680311730F2008730F3008F31C027B5
:1005A800803121002408FB002308FA0086313D260B
:1005B80080318F317B2780315F2B9F30F1002130D4
:1005C800F20020302000DB005B08F3005030DC0034
:1005D8005C08F4008F31D42780319F3086002130A9
:1005E80087007C30C03FC6308600213087007C30D1
:1005F8008100ED308600213087007C3081009F30FB
:100608002000D0002130D1006530DB005B08D2002B
:100618003F08D4003E08D3008731CB2780319F3074
:100628002000D0002130D1006930DB005B08D20007
:100638002830F1000030F2004F08F4004E08F300B3
:1006480087312727803172082000D4007108D30031
:100658008731CB2780319F302000D0002130D10056
:100668006F30DB005B08D2002830F1000030F20068
:100678003208F4003108F3008731272780317208E7
:100688002000D4007108D3008731CB2780319F30F8
:10069800F2002130F3008F31C02780318F317B2762
:1006A80080315F2B20004C086E3A03193A2A1E3A13
:1006B8000319E12A5F2B3000201CAB2B20102000EF
:1006C8000C17E0014A0860020318952B3208C30092
:1006D8003108C2004208DB004308DC000030DC1BA4
:1006E800FF30DD00DE005B08AF025C08B03B5D0850
:1006F800B13B5E08B23B4008DB004108DC0000303B
:10070800DC1BFF30DD00DE005B08AF075C08B03D96
:100718005D08B13D5E08B23D0130DB005B08E007D3
:10072800662B0C133109DB003209DC00DB0A0319E4
:10073800DC0A44085B07DD0045085C3DDE005D0817
:100748003000A30020005E083000A400111720002C
:100758000D1CD12B3F08803ADB0080305B02031D63
:10076800B72B03303E02031CBD2B20008E100E1544
:10077800132C20003F08803ADB007F305B02031D0A
:10078800C72BFE303E020318CD2B20008E140E1509
:10079800102C20008E140E11132C0E15CF1BF12BCC
:1007A8008E154F08803ADB0081305B02031DDE2B7B
:1007B80000304E020318EB2B20004F08803A803C93
:1007C800031DE92B4E08300028020318EE2B2000E9
:1007D8008E10142C20008E14142C8E144F08803A7E
:1007E800DB007F305B02031DFB2B02304E02031C33
:1007F8000F2C20004E09DB004F09DC00DB0A03192F
:10080800DC0A5C08803A803C031D0D2C5B08300034
:1008180028020318122C20008E11142C20008E158B
:10082800921FC0298E1092130100C029F1009C2C40
:1008380020300800703008005030080030300800C0
:100848007830080068300800583008004830080040
:1008580038300800743008006C3008006430080034
:10086800543008004C300800443008003430080088
:100878007A30080076300800723008006E300800C0
:100888006A30080066300800623008005A300800F4
:1008980056300800523008004E3008004A30080030
:1008A8004630080042300800363008003230080070
:1008B8007930080077300800753008007330080078
:1008C800713008006F3008006D3008006B30080088
:1008D8006930080067300800653008006330080098
:1008E80061300800593008005730080055300800BA
:1008F80053300800513008004F3008004D300800D0
:100908004B300800493008004730080045300800DF
:1009180043300800413008003930080037300800FB
:1009280035300800333008003130080071080800FD
:100938007108033A03191C2C073A03191E2C013AB3
:100948000319202C033A0319222C0E3A0319242CDC
:10095800013A0319262C033A0319282C013A0319E2
:100968002A2C073A03192C2C1D3A03192E2C033A6A
:100978000319302C013A0319322C063A0319342C86
:10098800033A0319362C013A0319382C0E3A031985
:100998003A2C383A03193C2C033A03193E2C013AF5
:1009A8000319402C073A0319422C013A0319442C25
:1009B800033A0319462C013A0319482C0E3A031935
:1009C8004A2C033A03194C2C013A03194E2C073AC6
:1009D8000319502C013A0319522C033A0319542CC9
:1009E800013A0319562C1D3A0319582C013A0319D8
:1009F8005A2C703A03195C2C073A03195E2C013AF9
:100A08000319602C033A0319622C013A0319642C68
:100A18000F3A0319662C013A0319682C033A031993
:100A28006A2C013A03196C2C073A03196E2C013A07
:100A38000319702C033A0319722C013A0319742C08
:100A48001C3A0319762C073A0319782C013A031932
:100A58007A2C033A03197C2C013A03197E2C0F3A9D
:100A68000319802C013A0319822C033A0319842CA8
:100A7800013A0319862C073A0319882C013A0319FD
:100A88008A2C033A03198C2C013A03198E2C3C3A10
:100A98000319902C073A0319922C013A0319942C44
:100AA800033A0319962C013A0319982C9A2C08003A
:100AB80020004609D0004709D100D00A0319D10AFD
:100AC8002500110820005007D20025001208200038
:100AD800513DD3005208BE005308BF00250012083C
:100AE8002000C700250011082000C6008030BE077E
:100AF8006930BF3D7C0A0319D22D0130D00050085F
:100B0800FC0702307C02031C08003F08803AD00032
:100B18007F305002031D922DFE303E02031CA02D93
:100B280020003F08803AD00080305002031D9E2DDF
:100B380003303E02031CA22DFC01FC0A4E30873113
:100B48006C27853120003E08CE073F08CF3D4F086F
:100B5800D1004E08D0000630D035D10D890BB02D0C
:100B68005008B9005108BA00890D893B8909BB00B2
:100B7800BC008731A027853120003A08C100390818
:100B8800C0007C0A031D08003108C4023208C53BB6
:100B98008F31EA272000CA01CA0A08003F08803AB4
:100BA800D0007F305002031DDB2DCE303E02031CE7
:100BB800080020003F08803AD00080305002031D12
:100BC800E72D33303E02031808004E3087316C277A
:100BD800853120003E08CE073F08CF3D4E08D000A3
:100BE8004F08D1000030D11BFF30D200D30050088D
:100BF800AA075108AB3D5208AC3D5308AD3D2A0841
:100C0800D0002B08D1002C08D2002D08D3000430C6
:100C1800D400D337D20CD10CD00CD40B0D2E4F08E6
:100C2800D6004E08D5000530D535D60D890B182EBF
:100C38005508D7005608D8000030D81BFF30D90017
:100C4800DA005708D0075808D13D5908D23D5A084C
:100C5800D33D5308BC005208BB005108BA005008E5
:100C6800B9008731A02720003A08C1003908C00020
:100C78000800FB1F482E2D308F316C278631FA096A
:100C8800FB09FA0A0319FB0A2000D1010A30F10016
:100C98000030F2007B08F4007A08F3008731272738
:100CA80086317108303E2000D0005108203E860071
:100CB8008701500881000130D0005008D1070A3060
:100CC800F1000030F2007B08F4007A08F300863166
:100CD8008F2686317208FB007108FA007B08803A7B
:100CE8002000D00080305002031D7C2E01307A0293
:100CF800031C8A2E4A2E01302000D1025108203EC2
:100D08008600870101088F316C2786312000510841
:100D1800031908007F2EF701F21F992EF109F20935
:100D2800F10A0319F20AF701F70AF41FA42EF309CE
:100D3800F409F30A0319F40A0130F5007508F706F7
:100D4800F801F901710872040319D32EF601F60AA5
:100D5800F21BB82E0130F135F20D890BAF2E0130A0
:100D6800F5007508F607AC2E0130F835F90D890B3A
:100D7800B92E72087402031DC32E71087302031C76
:100D8800CA2E7108F3027208F43B78140130F23667
:100D9800F10C890BCB2E0130F602031DB82E770813
:100DA8000319DB2EF809F909F80A0319F90A790871
:100DB800F2007808F10008000D340A3444344C3449
:100DC8003434593448344634203447345034533456
:100DD80044344F342034563431342E3431340D34C5
:100DE8000A34003420346C34703469343D340034AF
:100DF8002034703477346D343D34003420346C340E
:100E080070346F343D3400342034693431343D3427
:100E180000342034693432343D340034203478349A
:100E280078343D3400342034793479343D34003416
:100E3800643466343D340034723478343D340034DC
:100E480074343D340034F701F41F312FF309F409E9
:100E5800F30A0319F40AF701F70AF21F382FF10908
:100E6800F209F10A0319F20A7108720403195F2FD3
:100E7800F601F60AF21B4A2F0130F135F20D890B03
:100E8800412F0130F5007508F6073E2F72087402ED
:100E9800031D502F71087302031C562F7108F302AB
:100EA8007208F43B0130F236F10C890B572F0130F0
:100EB800F602031D4A2F77080319672FF309F4096F
:100EC800F30A0319F40A7408F2007308F100080021
:100ED800F400740886008701403FF100413FF200AA
:100EE8007208803AF300FD307302031D7D2F013034
:100EF8007102031C862F7408860087010030C03FEA
:100F08007D30C13F740886008701403FF100413FB2
:100F1800F2007208803AF30003307302031D962F23
:100F28000030710203180800740886008701003039
:100F3800C03F8330C13F08002000BC1BB62F3C08CF
:100F4800031DAD2F3B08031DAD2F80303A02031C53
:100F5800B62F0030BC000030BB007F30BA00FF3035
:100F6800B9000800BC1F08000130390280303A3B44
:100F7800FF303B3BFF303C3B03180800FF30BC0010
:100F8800FF30BB008030BA000130B90008002730BC
:100F98002000D3070030D43DD41FD42FD301D4016F
:100FA8005408803AF80080307802031DDD2F4F3056
:100FB8005302031CE42F4E302000D3000030D4002D
:100FC800200053085007F8005408513DF9007808EC
:100FD80086007908870052088100080064008001B3
:100FE80001310130FE020030FF3B7F087E04031907
:040FF8000034F32F9F
:101ED800F10023009E1C6D2F71089A0008000F3036
:101EE80021009F0001309D00A0309E0008000D30A9
:101EF8008F316C278F310A308F316C270800F3003F
:101F08000130F102710A031908007308860087017D
:101F180081010130F2007208F307842F1830230082
:101F28009F0004309E0010309D0013309B009D17C9
:101F38009E1621001112911208002000911EA72F51
:101F480023001908080023009D1CAE2F1D12000055
:101F580023001D16003008001A302000C800063083
:101F6800C9000130C8020030C93B480A031DB52F1B
:101F7800490A03190800B52F720884007308850000
:101F8800120003190800720884007308850000080D
:101F98008F316C278F310130F2070030F33DC02FAD
:101FA8000130F402740A0319E42F710886007208DC
:101FB8008700730881000130F1070030F23DD42F0B
:101FC8007108860072088700810108002000C0019E
:101FD800C101CE01CF010030AD000030AC000030AF
:101FE800AB000030AA000030B2000030B100003071
:081FF800B0000030AF0008004A
:020000040001F9
:04000E00C7EFFFFF3A
:10E0000002000000000000002000500046004F0009
:10E0100064006C0034007900680066002E00000087
:00000001FF
